:100000000C9415010C9432010C9432010C943201C1
:100010000C9432010C9432010C9432010C94320194
:100020000C9432010C9432010C9432010C94320184
:100030000C9432010C9432010C9432010C94320174
:100040000C9432010C9432010C9451010C947901FE
:100050000C9432010C9432010C9432010C94320154
:100060000C9432010C9432012B4154455849540DE3
:100070000A002B4F4B0D0A002B61746174002B4159
:10008000544154002B4F4B0D0A004552520D0A00AB
:1000900041542B424C0041542B5354520041542B99
:1000A000474F544F0041542B434C520041542B4274
:1000B0004155440041542B4543484F004465627507
:1000C00067446973706C61792076312E302028483E
:1000D0006F626269656C656B74726F6E696B612EBD
:1000E00068752C20627920546F7069290D0A0041CF
:1000F000542B5645523F0041542B424C205B302D2F
:100100003235355D202D2053657420646973706C21
:100110006179206261636B6C6967687420627269DF
:100120006768746E6573730D0A0041542B53545203
:1001300020737472202D205072696E742073747253
:10014000696E670D0A0041542B474F544F207820A9
:1001500079202D20476F746F2058590D0A004154A3
:100160002B434C52202D20436C65617220646973CF
:10017000706C61790D0A0041542B42415544205B5B
:10018000302D335D20536574206261756472617433
:10019000652028303D393630302C20313D31393220
:1001A00030302C20323D35373630302C20333D3145
:1001B0003135323030290D0A0041542B4543484F28
:1001C000205B302F315D202D204563686F206F66E6
:1001D000662F6F6E0D0A0041542B5645523F202D5D
:1001E00020446973706C6179206E616D6520616E69
:1001F000642076657273696F6E20696E666F0D0A92
:10020000000D0A2D2D2D2D2D2D2D2D2D2D2D2D2D8E
:100210002D2D2D2D2D2D2D2D2D2D0D0A003F004185
:10022000542B48454C500041540011241FBECFEFC1
:10023000D4E0DEBFCDBF11E0A0E0B1E0EEECFBE02A
:1002400002C005900D92AC31B107D9F712E0ACE1D4
:10025000B1E001C01D92A532B107E1F70E9456043A
:100260000C94E5050C9400009B01AC0160587B47A1
:10027000814E9F4FF3E0660F771F881F991FFA95F5
:10028000D1F7E4E0220F331F441F551FEA95D1F741
:100290000E94BA05215030402093C4003093C5001D
:1002A00008951F920F920FB60F9211248F939F9370
:1002B000EF93FF938091C0009091C6008C7181F400
:1002C0008091A001E82FF0E0E25EFE4F90838F5F07
:1002D0008093A0018091A001803410F01092A001C1
:1002E000FF91EF919F918F910F900FBE0F901F90F4
:1002F00018951F920F920FB60F9211248F939F9310
:10030000EF93FF939091A3018091A1019817C1F001
:100310008091C00080648093C0009091A101E92F7A
:10032000F0E0EB55FE4F80818093C6009F5F909375
:10033000A1018091A10187FF08C01092A10105C011
:100340008091C1008F7D8093C100FF91EF919F91BB
:100350008F910F900FBE0F901F9018959091A00154
:1003600080915F01981711F4E0E010C080915F0167
:10037000E82FF0E0E25EFE4FE0818F5F80935F0147
:1003800080915F01803410F010925F018E2F0895EC
:100390009091A301E92FF0E0EB55FE4F80839F5F22
:1003A0009093A3018091A30187FF02C01092A30143
:1003B0008091C10080628093C1000895CF93DF9344
:1003C000EC0103C021960E94C80188818823D1F7DF
:1003D000DF91CF910895CF93DF93EC01FE018491DB
:1003E000882321F00E94C8012196F8CFDF91CF9198
:1003F00008951F93182F64E60E949A05805D0E945D
:10040000C801812F64E60E949A05192F892F6AE09E
:100410000E949A05805D0E94C801812F6AE00E94B7
:100420009A05892F805D0E94C8011F9108959091BF
:10043000A3018091A1019817D1F70895519A50987E
:1004400088E98093C10086E08093C2008091C60055
:100450008091C00087FDFACF80EC8093C00080912E
:10046000C6001092A00110925F011092A401109298
:10047000A3011092A10160E875E280E090E00E9483
:100480003401089520E43CE904C0F9013197F1F703
:1004900081508823D1F70895FC0120E03AE00DC097
:1004A0009D3071F09A3061F0903251F0239F802D91
:1004B0001124292F2053280F31969081992381F7F9
:1004C000822F08951F93182F64E60E949A05805D7D
:1004D0000E94C801812F64E60E949A05192F892F76
:1004E0006AE00E949A05805D0E94C801812F6AE03F
:1004F0000E949A05892F805D0E94C8011F9108956E
:10050000EF92FF920F931F93DF93CF93CDB7DEB798
:1005100028970FB6F894DEBF0FBECDBF8091600163
:10052000882309F428C1FE013196CE010996119263
:10053000E817F907E1F700E611E020E030E0BE013E
:100540006F5F7F4F422FF80191918F01892F815664
:100550008A3108F49052992379F0903269F09D33F2
:1005600059F0FB01E20FF31F90834F5F2F5F3F4F66
:10057000F1E007361F0731F7FE01E40FF11D11828C
:10058000F8018081803211F08D3311F40F5F1F4F1D
:100590007E010894E11CF11CC70167E272E00E9431
:1005A000DC05892B09F4E3C0C7016FE172E00E940A
:1005B000DC05892B41F0C7016DE172E00E94DC058A
:1005C000892B09F051C081E092E00E94EB019091EB
:1005D000A3018091A1019817D1F787ED91E00E94C6
:1005E000EB019091A3018091A1019817D1F789EBBC
:1005F00091E00E94EB019091A3018091A1019817D5
:10060000D1F787E791E00E94EB019091A3018091DF
:10061000A1019817D1F78EE591E00E94EB0190912E
:10062000A3018091A1019817D1F786E491E00E947F
:10063000EB019091A3018091A1019817D1F78AE273
:1006400091E00E94EB019091A3018091A101981784
:10065000D1F787EF90E00E94EB019091A301809188
:10066000A1019817D1F783C0C7016FEE70E00E9417
:10067000DC05892B19F48CEB90E077C0C70164EBA3
:1006800070E00E94DC05892B61F4C8010E944C02D5
:1006900010921C01813309F06AC081E080931C0133
:1006A00066C0C7016CEA70E00E94DC05892BF9F492
:1006B000C8010E944C02823049F0833061F08130E1
:1006C00079F460E07BE480E090E00EC060E071EEE1
:1006D00080E090E009C060E072EC81E090E004C04E
:1006E00060E875E280E090E00E94340140C0C701FC
:1006F00065EA70E00E94DC05892B19F40E94290547
:1007000036C0C7016DE970E00E94DC05892B99F4C1
:10071000C8010E944C02F82E01C08F01F80181919E
:1007200080538A30D0F3CF010E944C02682F8F2D66
:100730000E941D051CC0C70166E970E00E94DC052F
:10074000892B21F4C8010E94460511C0C70160E948
:1007500070E00E94DC05892B31F4C8010E944C0234
:100760008093B40004C08AE890E00E94EB0184E822
:1007700090E00E94EB0128960FB6F894DEBF0FBE02
:10078000CDBFCF91DF911F910F91FF90EF90089512
:100790001F939091A00180915F01981709F466C0A2
:1007A0000E94AE01182F80911C01882319F0812F1F
:1007B0000E94C8011D3091F580E691E06EE770E07F
:1007C0000E94DC05892B41F080E691E068E770E04B
:1007D0000E94DC05892B49F482E790E00E94EB013E
:1007E00081E080931D011092600180911D0188239A
:1007F00071F46091A2010E941D0580E691E00E94C3
:1008000046058091A2018F5F8093A20102C00E94E1
:10081000800210925E011092600128C01B3199F491
:100820000E9429051092600110925E011092A201AF
:1008300080911D018823D1F088E690E00E94EB01B1
:1008400010921D0113C0103288F080915E018F3329
:1008500068F4E82FF0E0E05AFE4F1083E82FEF5FD6
:10086000E0935E01F0E0E05AFE4F10821F91089580
:10087000539A0E941E0283E28093B00084E080932A
:10088000B10088EC8093B4008CE00E9460050E9467
:1008900029050E942905789481E080931C0110921B
:1008A0005E011092A20110921D0108950E94380469
:1008B00080E060E00E941D0580E091E00E94460516
:1008C00080E061E00E941D0580E191E00E94460504
:1008D00022E340E45CE903C0CA010197F1F721502B
:1008E000D8F70E94C803FDCF662311F02A9A01C0F1
:1008F0002A982998549A559A569A579A5F985E98CA
:100900005D985C9887FD5F9A86FD5E9A85FD5D9A8D
:1009100084FD5C9A289A00C028985F985E985D983C
:100920005C9883FD5F9A82FD5E9A81FD5D9A80FDF1
:100930005C9A289A00C028985C9A5D9A5E9A5F9AA1
:100940000895882311F02A9A01C02A98299A549868
:10095000559856985798289A00C04C9B02C080E141
:1009600001C080E04D9980624E9980644F99806803
:10097000289800C0289A00C04C9981604D998260E7
:100980004E9984604F9988602898089580E00E946D
:10099000A10487FDFBCF88E090E00197F1F780E0AC
:1009A0000E94A10408951F93182F0E94C604812F4E
:1009B00060E00E9474041F9108951F93182F0E94F5
:1009C000C604812F61E00E9474041F9108950F9363
:1009D0001F938C0168EE73E00E94A605862F805D50
:1009E0000E94DD04C80168EE73E00E94A605182F7E
:1009F000092F64E670E00E94A605862F805D0E94A4
:100A0000DD04812F902F64E670E00E94A605182F68
:100A1000092F6AE070E00E94A605862F805D0E9483
:100A2000DD04812F902F6AE070E00E94A605805DB2
:100A30000E94DD041F910F910895662311F48058E0
:100A400001C080540E94D30408950E94C60490E01F
:100A5000089581E00E94D304089582E00E94D304A7
:100A600008951F93182F0E94C6041A3049F4803449
:100A700010F080E001C080E480580E94D30404C0DC
:100A8000812F61E00E9474041F910895CF93DF933A
:100A9000EC0102C00E94310589918823D9F7DF91CA
:100AA000CF910895CF93DF93EC0102C00E943105EE
:100AB000FE01219684918823C9F7DF91CF91089593
:100AC0001F93182F229A219A209A549A559A569A2F
:100AD000579A80E09AEF0197F1F75D9A5C9A289A0D
:100AE00000C0289880E09EE40197F1F7289A00C0A2
:100AF000289880E091E0FC013197F1F7289A00C036
:100B00002898FC013197F1F75C98289A00C0289842
:100B10000197F1F788E20E94D30488E00E94D30491
:100B20000E94290586E00E94D304812F0E94D304ED
:100B30001F910895991B79E004C0991F961708F03A
:100B4000961B881F7A95C9F780950895AA1BBB1B31
:100B500051E107C0AA1FBB1FA617B70710F0A61BBD
:100B6000B70B881F991F5A95A9F780959095BC01DE
:100B7000CD010895A1E21A2EAA1BBB1BFD010DC0D9
:100B8000AA1FBB1FEE1FFF1FA217B307E407F5073D
:100B900020F0A21BB30BE40BF50B661F771F881F19
:100BA000991F1A9469F760957095809590959B01AF
:100BB000AC01BD01CF010895FB01DC018D910590D1
:0E0BC00080190110D9F3990B0895F894FFCF16
:100BCE004465627567446973706C61792076310093
:0C0BDE0020202020627920546F706900F4
:00000001FF
